S113020083860097109740974186EE97113F458368
S1130210BD032B7C00409640BDF64EBDF7ADBD033B
S1130220708150240220073F2183860097403FC3FA
S1130230D061C3F04ACC0BFF83CE00039611BDF608
S11302404EBDF7AD0C8248250220EE96110C82209B
S1130250240ACE000ABD030B250720DDBD0320249C
S1130260DB3F0272FB7B830101013FC3C85EC3D045
S11302705BC3D8518F000283CE0003BD030B240E51
S11302803FC3EC93D3080DC3E84A837E021396114F
S1130290BDF64EBDF7AD97413F8F0003839611B174
S11302A0004126EA9641163F8F0002D3C803D3D0FB
S11302B003C3D8718F000283CE0003BD030B240E49
S11302C03FC3E800D3080DC3EC4A837E02139611A2
S11302D0BDF64EBDF7AD97413F8F0003839611B134
S11302E0004126EA96411024113FC3F035D308108B
S11302F0C3F04AC3D061837E02103FC3F05FD308CA
S113030010C3F04AC3D061837E0210BDF64E96112D
S1130310BDF7AD0C8220250139BD032025FA20EE5E
S11303200C0926010D3F8F000383393F428F0002E1
S113033083CE0800BDF64EB6C240BDF7AD0C82A018
S113034024080926EFCE00030D393F8F000472FD07
S1130350468F000483BDF64EB6C240BDF7AD0C8295
S1130360A02408BD032020ED010101390101010190
S10903703F8F00108339E9
